:100000003BC1000055C1000053C1000051C10000B8
:100010004FC100004DC100004BC1000049C10000AC
:1000200047C1000045C1000043C100000C94D10D40
:100030003FC100003DC100003BC100000C94840999
:1000400037C1000035C1000033C100008CC300007F
:100050002FC100002DC100002BC1000085C1000090
:1000600027C1000025C1000023C1000021C10000FC
:100070001FC100001DC100001BC1000019C100000C
:1000800017C1000015C1000013C1000011C100001C
:100090000FC100000DC10000120110010200000894
:1000A000EB034B20010001020002040309041803C2
:1000B0004400650061006E002000430061006D0097
:1000C00065007200610000002E034C0055004600E0
:1000D000410020005500530042002D005200530003
:1000E00032003300320020004100640061007000E3
:1000F000740065007200000012011001FF0000088A
:10010000EB030421000201020302040309040C03AF
:10011000410054004D0045004C0000001803410010
:100120005600520049005300500020006D006B0043
:1001300049004900000009000A000A000B000C00F9
:100140000D000D000E000F00100010001200130033
:100150001300140016001600180019001A001C00E5
:100160001D001F0020002200230025002700290079
:100170002B002E0030003200340037003A003D00E2
:100180004000430046004A004E00520055005A000D
:100190005E00630068006D00730078007E008400DC
:1001A0008B0091009900A000A900B100B900C30024
:1001B000CC00D600E100EC00F700040111011E01A3
:1001C0002D013B014B015B016C017D019101A501FA
:1001D000BA01CF01E601FE01160231024C026A02A9
:1001E0008802A802CA02ED021103380360038B03E0
:1001F000B803E70318044B048104B904F50434057B
:100200007505B90501064E069D06EF064807A307CA
:1002100004086508D0084009B6092B0AAB0A300B60
:10022000C30B510CEE0C8F0D400EF60EAF0F681085
:1002300047111412F512ED13E214F015F9161B18FC
:100240005C19911AE51B251D831E0320AB21302369
:1002500032250F27F128F82A1A2D492FA1311434FD
:10026000A1364539173C1A3F34426045DF48704C8F
:10027000400041014243030011241FBECFEFD4E0F0
:10028000DEBFCDBF11E0A0E0B1E0E8E8F2E202C0DD
:1002900005900D92A23CB107D9F712E0A2ECB1E0B3
:1002A00001C01D92AC3EB107E1F752D10C9442114E
:1002B000A7CEFC018FB7F894718360837383628348
:1002C00075836483640F751F7783668351874087C6
:1002D000138612868FBF0895CF93DF93EC01E881D8
:1002E000F9816083888199810196998388832E8121
:1002F0003F818217930721F48C819D8199838883A4
:100300002FB7F8948A859B8501969B878A872FBF94
:10031000DF91CF910895CF93DF93EC01EA81FB81C8
:100320003191FB83EA838E819F81E817F90721F4DD
:100330008C819D819B838A832FB7F8948A859B85C6
:1003400001979B878A872FBF832FDF91CF910895D5
:100350005E9A08955E980895FC01208920FF02C0EE
:100360005F9808955F9A08951F920F920FB60F92AB
:1003700011242F933F934F935F936F937F938F93AA
:100380009F93AF93BF93EF93FF936091CE008EB393
:10039000843089F48FB7F8942091590230915A0231
:1003A0008FBF80915702909158022817390719F092
:1003B0008FE492E091DFFF91EF91BF91AF919F9118
:1003C0008F917F916F915F914F913F912F910F90FE
:1003D0000FBE0F901F9018951F93FC01818D8130E7
:1003E00019F0823019F404C010E303C010E001C01A
:1003F00010E2808D823009F41860828D873031F0F0
:10040000883031F0863029F4126003C0146001C0D6
:1004100016605B9A1092C9001092C8001092CA0030
:100420002489358946895789CA01B90196958795E6
:100430007795679560587B47814E9F4F0E940611C4
:10044000215030403093CD002093CC001093CA004F
:1004500082E08093C80088E98093C9005B981F916F
:100460000895FC018091C201882311F4CF0108C1D5
:10047000CF0137C18091C201882321F480E091E04F
:100480000C94581008951F938091C2018823A9F4F9
:1004900080E091E00E943110182F117083EC91E000
:1004A0006FEC71E040E850E004DF8FE492E06BE530
:1004B00072E040E850E0FDDE07C082E060E842E321
:1004C0000E94EE0C182F1170112311F05E9A01C0DA
:1004D0005E981F91089584B7877F84BF88E10FB627
:1004E000F89480936000109260000FBEE0EDF0E0A1
:1004F000808185608083E1E6F0E080E8808310827F
:100500003D98459A00000000000086B182958695CE
:100510008770809581708093C2015F9A579A84B1E9
:10052000817E84B98AB180678AB98BB180678BB9C3
:100530000C94C20D8EB3843051F482E08093E900B4
:100540008091E80082FF03C05E9822D15E9A0895F0
:100550001F93CF93DF93BFDF8091C201882379F48B
:1005600083EC91E06FEC71E040E850E0A2DE8FE4B4
:1005700092E06BE572E040E850E09BDE01C015D2EE
:100580007894C0E0D0E08091C201882309F06BC06C
:100590008FB7F8942091CD013091CE018FBF80911B
:1005A000CB019091CC012817390769F080E091E0E8
:1005B0000E949B0FBC0197FD06C05C9883EC91E004
:1005C0008BDEC0E0D0E08FB7F894209159023091D3
:1005D0005A028FBF2115310529F15D9880910101E3
:1005E0008F708093E9008091E80080FF19C0C901F5
:1005F0002031310510F08FE090E0182F0FC0E0910E
:100600005102F091520280E091E060810E940C1052
:100610001150882329F48FE492E07DDE112379F7CD
:10062000C0E0D0E08091C80085FF13C02FB7F894D8
:100630008091CD019091CE012FBF892B51F083EC99
:1006400091E069DE982F8091C80085FFFCCF9093E0
:10065000CE0080E091E00E94F50F199B02C05E98E9
:1006600003C05E9A01C066DF0E94870F219683E077
:10067000C83ED80709F087CF8BB180638BB981CF93
:10068000DA01F9011082923049F0933069F091302B
:1006900001F5E8E9F0E022E130E01FC09083EBE1F2
:1006A000F1E02EE330E019C0813049F0813018F0DC
:1006B000823079F408C0EAEAF0E0849107C0EEEAFB
:1006C000F0E0849103C0E8ECF0E08491282F30E062
:1006D00004C0E0E0F0E020E030E0ED93FC93C901DD
:1006E0000895DA01F9011082923049F0933069F0EF
:1006F000913089F5E8EFF0E022E130E030C09083FE
:10070000E9E5F1E020E230E02AC0813059F08130A3
:1007100028F0823059F08330F1F40EC0EAE0F1E0C5
:10072000849107C0EEE0F1E0849103C0ECE1F1E0D8
:100730008491282F30E013C080917901282F30E078
:1007400082E390E0909388018093870182E0808328
:10075000E9E7F1E004C0E0E0F0E020E030E0ED9314
:10076000FC93C901089578941F920F920FB60F92CF
:1007700011248F938AB5882321F08AB581508ABDD0
:1007800001C015BC8F910F900FBE0F901F90189550
:10079000FF920F931F931091F10084E68ABD85E0CC
:1007A00085BD133109F4C0C01431F0F4163009F4DA
:1007B00080C0173048F4113099F1113008F4CBC0E3
:1007C000143008F0C8C049C0103109F4A9C0113173
:1007D00020F41A3009F0BFC091C0113109F4A2C051
:1007E000123109F0B8C0A6C0183109F4A5C01931FA
:1007F00068F4153109F498C0153108F498C0163121
:1008000009F495C0173109F0A6C099C01D3120F434
:100810001A3108F091C093C01D3109F09CC092C0FC
:100820008091E8008B778093E80082E08093E90074
:100830008091EC0081608093EC001093F1001092A5
:10084000F1008AE08093F10087E991E06AE070E0CE
:1008500040E050E00E949C0C94C00091F1001230E6
:1008600011F0FF2402C0F090F1008091E8008B7736
:100870008093E80082E08093E9008091EC00816041
:100880008093EC001093F100802FAFD0123041F430
:1008900081FF0DC01092F100802F6F2DAED071C07E
:1008A00080FF05C01092F100802F97D068C080ECC7
:1008B00066C08EED92E064E070E040E050E098D7D2
:1008C0008091E8008B778093E80082E08093E900D4
:1008D0008091EC0081608093EC008091DE02909129
:1008E000DF02A091E002B091E102B7FF03C081E016
:1008F0008093DD0286E08093F1000FC08091E800D4
:100900008B778093E80082E08093E9008091EC008F
:1009100081608093EC001093F1001092F10031C0DF
:1009200058D434C023D432C0812FF3D22FC0812FAA
:1009300046D22CC0F6D12AC0812FF1D027C0812FFA
:10094000A9D024C056D122C08091E8008B77809333
:10095000E8000E945D0D8091F2008034A9F380913F
:10096000E8008B778093E80082E08093E900809133
:10097000EC0081608093EC001093F10089EC80938F
:10098000F1008091E8008E778093E80015BC0E940A
:100990005D0D82E08093E9008091EC008E7F809372
:1009A000EC001F910F91FF9008958BE987BD82E0C5
:1009B00084BD80936E0039D0D7C4982FE2EAF1E06D
:1009C0008081981741F081E0ED3BF80711F03396F4
:1009D000F7CFE0E0F0E0CF010895EFDFFC010097F2
:1009E00011F480E0089582810895E7DFFC0100970B
:1009F00011F480E00895818108950F931F93182FBB
:100A0000062FDBDFFC01009769F002831E3919F421
:100A100080E090E004C0183929F481E090E0602F74
:100A20000E9430111F910F9108950F931F9380E042
:100A300090E00E942811182F81E090E00E94281178
:100A4000082F1F3F21F08EE9B8DFFC0112830F3F12
:100A500021F088E9B2DFFC0102831F910F91089514
:100A6000282F40EA5FE003C0CA010197F1F7222373
:100A700021F08AB521508823B9F70895982F8091E5
:100A8000C001882329F09EBD0DB407FEFDCF089557
:100A9000892FAAC4DF92EF92FF920F931F93DF93E7
:100AA000CF9300D000D0CDB7DEB7D82E8E010F5F28
:100AB0001F4FC80164E070E040E050E0EBD6809149
:100AC000E8008B778093E80082E08093E9008091D2
:100AD000EC0081608093EC0085E0E82EF12CEC0EB8
:100AE000FD1EF80181918F01C9DF0E151F05C9F7A1
:100AF000D092F1001092F1001092F1008091E80084
:100B00008E778093E8000F900F900F900F90CF9109
:100B1000DF911F910F91FF90EF90DF900895BF92AA
:100B2000CF92DF92EF92FF920F931F93DF93CF93B9
:100B3000CDB7DEB729970FB6F894DEBF0FBECDBF95
:100B4000B82ECE01059665E070E040E050E0A2D6F8
:100B50008091E8008B778093E80082E08093E90041
:100B60008091EC0081608093EC008E010A5F1F4F42
:100B70007E010894E11CF11C9AE0C92ED12CCC0E08
:100B8000DD1EF80190818091C001882331F09EBD67
:100B90000DB407FEFDCF8EB502C0892F25D4F70115
:100BA00081937F010F5F1F4F0C151D0551F7B09208
:100BB000F1001092F1008D81FE01E80FF11D80819E
:100BC0008093F1001092F1008091E8008E7780937D
:100BD000E80029960FB6F894DEBF0FBECDBFCF91C7
:100BE000DF911F910F91FF90EF90DF90CF90BF901A
:100BF0000895EF92FF920F931F93DF93CF93CDB79A
:100C0000DEB7C250D1400FB6F894DEBF0FBECDBFE5
:100C1000CE01019663E070E040E050E03BD634E066
:100C2000E32EF12CEC0EFD1E6981C70170E040E05F
:100C300050E030D68091E8008B778093E80082E026
:100C40008093E9008091EC0081608093EC008DE15D
:100C50008093F1001092F10000E00BC08981081729
:100C600028F4F701E00FF11D808101C080E006DF6C
:100C70000F5F8B81081790F310E024E0E22EF12C37
:100C8000EC0EFD1E2BC089819091C001081778F4ED
:100C9000F701E00FF11D8081992331F08EBD0DB475
:100CA00007FEFDCF8EB501C09FD30F5F0AC0992309
:100CB00031F01EBC0DB407FEFDCF8EB502C080E042
:100CC00093D38093F1008091E80085FD06C0809168
:100CD000E8008E778093E800F0D61F5F8A811817AE
:100CE00090F21092F1009091E8008091E8008E77E8
:100CF0008093E80095FD07C0E0D68091E8008E77EC
:100D00008093E800DAD6CE5FDE4F0FB6F894DEBFF0
:100D10000FBECDBFCF91DF911F910F91FF90EF904C
:100D20000895EF92FF920F931F93DF93CF9300D01C
:100D300000D000D0CDB7DEB7CE01019666E070E0FE
:100D400040E050E0A7D58091E8008B778093E800E1
:100D500082E08093E9008091EC0081608093EC0058
:100D60008E010D5F1F4F47E0E42EF12CEC0EFD1EAF
:100D7000F80181918F0182DE0E151F05C9F78A8166
:100D8000882321F489816CDE90E002C058D3982F2B
:100D900082E18093F1009093F1008091E8008E77DA
:100DA0008093E80026960FB6F894DEBF0FBECDBF45
:100DB000CF91DF911F910F91FF90EF900895DF92F7
:100DC000EF92FF920F931F93DF93CF9300D00F9278
:100DD000CDB7DEB7F82ECE01019663E070E040E0BB
:100DE00050E058D599818A8189839A838091E8005F
:100DF0008B778093E80082E08093E9008091EC009B
:100E000081608093EC00F092F1001092F10000E01C
:100E100010E068E0D62EEE24E39458C08091DD0205
:100E2000882319F02AD31092DD028B8127DE80916E
:100E3000DE029091DF02A091E002B091E102892FE1
:100E40009A2FAB2FBB271ADE8091DE0217DE80912E
:100E5000C001882331F01EBC0DB407FEFDCF8EB556
:100E600002C080E0C1D28093F1008091E80085FD4E
:100E700006C08091E8008E778093E8001ED624E1BA
:100E8000F21619F48B818D258B8300FD03C086E15A
:100E9000F816D1F48091DE029091DF02A091E00279
:100EA000B091E1020196A11DB11D8093DE029093E5
:100EB000DF02A093E002B093E10226E1F21621F0F6
:100EC000892B11F4E092DD020F5F1F4F89819A8117
:100ED0000817190708F4A2CF1092F1009091E800CA
:100EE0008091E8008E778093E80095FD07C0E5D5F6
:100EF0008091E8008E778093E800DFD50F900F9007
:100F00000F90CF91DF911F910F91FF90EF90DF90A5
:100F100008954F925F926F927F928F929F92AF92BD
:100F2000BF92CF92DF92EF92FF920F931F93DF93C6
:100F3000CF93CDB7DEB7C950D1400FB6F894DEBF1E
:100F40000FBECDBF182FCE01019669E070E040E0E2
:100F500050E0A0D46A81798181E06130780798F00F
:100F60008091E8008B778093E80082E08093E9002D
:100F70008091EC0081608093EC001093F10080EC94
:100F80008093F100D6C07A836983CE010A9640E04F
:100F900050E080D489819A810A968F739070892B52
:100FA00031F48091E8008B778093E80086D58091BA
:100FB000E8008B778093E80082E08093E9008091DD
:100FC000EC0081608093EC00133111F4888401C03F
:100FD00089846090DE027090DF02EE24FF24FAE044
:100FE000AF2EB12CAC0EBD1ECC24DD24E8E04E2E7D
:100FF000552453946DC0F50190800B818091DD02E2
:10100000882319F03AD21092DD028D8137DD80916C
:10101000DE029091DF02A091E002B091E102892FFF
:101020009A2FAB2FBB272ADD8091DE0227DD892D89
:1010300025DD133119F48D8184258D83E114F104AC
:1010400081F4981471F0C0FE05C0133119F48F813A
:10105000886002C08F81877F8F83E090DE02F090EE
:10106000DF0200FD12C0E114F10421F403FD02C00F
:10107000097F0260802FB701482D2C810F8106D295
:10108000282F882361F5EE24FF24C0FC02C015310F
:10109000C9F48091DE029091DF02A091E002B0914C
:1010A000E1020196A11DB11D8093DE029093DF0243
:1010B000A093E002B093E102133121F4892B11F4E3
:1010C0005092DD020894A11CB11C0894C11CD11CD3
:1010D00089819A81C816D90608F48DCF20E08B81CA
:1010E00087FF23C08E81CADC872DC8DC862DC6DC35
:1010F00080E0C4DC8B8185FF06C0E114F10419F4A3
:101100008F7C80618B838B81B701482D2C810F816F
:10111000BDD1282F133149F48091DE029091DF0276
:10112000892B19F481E08093DD021093F100209364
:10113000F1008091E8008E778093E800C75FDE4F72
:101140000FB6F894DEBF0FBECDBFCF91DF911F91D8
:101150000F91FF90EF90DF90CF90BF90AF909F9056
:101160008F907F906F905F904F9008950F931F9393
:10117000DF93CF9300D0CDB7DEB7CE01019662E00A
:1011800070E040E050E086D308EE10E0F801808186
:101190008B77808382E08093E900ECEEF0E0808141
:1011A0008160808389815CDC80E0B7D1F1D08A8165
:1011B00057DCE1EFF0E081E180831082F80180816B
:1011C0008E7780830F900F90CF91DF911F910F91B9
:1011D00008958F929F92AF92BF92CF92DF92EF923B
:1011E000FF920F931F93DF93CF93CDB7DEB72F9767
:1011F0000FB6F894DEBF0FBECDBFCE0105966BE0F3
:1012000070E040E050E046D38091E8008B77809317
:10121000E80082E08093E9008091EC008160809397
:10122000EC001092DE021092DF021092E0021092A7
:10123000E1028F8115DC7DD181E06FD18E8110DCE0
:10124000BCE08B2E912C8C0E9D1E5E010894A11C7F
:10125000B11CA0E1CA2ED12CCC0EDD1E2AC089857E
:10126000FFDBF80190818091C001882331F09EBDA1
:101270000DB407FEFDCF8EB502C0892FB5D0F701A2
:1012800081937F010F5F1F4F0C151D0541F78B8563
:101290008823D1F0FE01E80FF11D90818A8598170F
:1012A00099F080E03AD18E81DBDB81E036D18E810E
:1012B000D7DB9885992351F08AB5882339F091506E
:1012C000988784017501CBCF90E001C090EC80E15C
:1012D0008093F1009093F1008091E8008E778093E5
:1012E000E8002F960FB6F894DEBF0FBECDBFCF91AA
:1012F000DF911F910F91FF90EF90DF90CF90BF9003
:10130000AF909F908F9008951F920F920FB60F92FB
:1013100011248F93199908C08091DB0287FF02C0C6
:101320002A9A1BC02A9819C08091DB02880F8093EB
:10133000DB028091DC0281508093DC028091DC0230
:10134000882321F41092810082E086BB1B9B05C09C
:101350008091DB0281608093DB02199A8F910F905C
:101360000FBE0F901F9018953E9A10926F0010922A
:1013700085001092840081E090E090938900809332
:10138000880080E48093800089E080938100089544
:101390008091C001882349F084B1897F84B985B1E7
:1013A000867F85B91CBC1DBC089584B1897F84B932
:1013B00085B1867F85B9D8CF92E090936F00109267
:1013C000850010928400E82FF0E0EE0FFF1FE85D2B
:1013D000FE4F85919491909389008093880010929C
:1013E00080001092810008958093DB0288E0809352
:1013F000DC028091DB0287FF02C02A9A01C02A9892
:1014000010928500109284008AE080938100809180
:10141000DC02882319F08AB58823C9F7109281006D
:101420008091DB020895982F8091C001882329F0D4
:101430009EBD0DB407FEFDCF0895892FD5CF80EF57
:10144000F2DF80E0F0DF80E0EEDF8091C0018823F2
:1014500031F01EBC0DB407FEFDCF8EB502C080E09A
:10146000C3DF80FF03C08AB5882349F78AB5882384
:1014700011F481E8089580E008958DE4D4DF80E0E0
:10148000D2DF8091E002CFDF80E0CDCFEF92FF92FC
:101490000F931F937B01142F90E08E778830910576
:1014A00081F18930910534F48230910559F0049727
:1014B00059F50BC08032910541F08034910509F156
:1014C000409711F5822FCCDA1FC0802FACDF8F2D13
:1014D000AADF8E2DA8DF8091C001882331F01EBCC9
:1014E0000DB407FEFDCF8EB502C080E07DDF811711
:1014F00019F48AB5882349F78AB5882329F490E836
:1015000004C09DDF982F01C090E084E68ABD892F3A
:101510001F910F91FF90EF900895882339F0249A3E
:101520008EE95BDA882319F42C9A089524982C9874
:10153000089588E952DAE82F8730D8F481E0809363
:10154000C001F0E0E059FD4FE491E061209A289A53
:1015500084B1866084B923982B9AE6FF03C08DB5C9
:10156000816002C08DB58E7F8DBD2098E064ECBD9A
:1015700008951092C00184B1866084B985B18960F4
:1015800085B98E2F19CF9C014091EA025091EB0250
:101590004617570718F4F90190E03CC06115710532
:1015A00011F0AB01F8CF8091E8008E778093E800CE
:1015B00040E050E0F0CF8EB3882309F440C085307E
:1015C00009F43FC08091E80083FD3DC08091E800B0
:1015D00082FD2FC08091E80080FF1CC08091F20046
:1015E000282F30E007C081918093F1004150504096
:1015F0002F5F3F4F4115510519F02830310598F301
:1016000090E02830310509F491E08091E8008E7770
:101610008093E8004115510571F6992361F609C0E0
:101620008EB3882361F0853061F08091E80083FDFE
:101630000AC08091E80082FFF3CF80E0089582E045
:10164000089583E0089581E008959C014091EA02A5
:101650005091EB024617570718F4F90190E03DC08E
:101660006115710511F0AB01F8CF8091E8008E771C
:101670008093E80040E050E0F0CF8EB3882309F477
:1016800041C0853009F440C08091E80083FD3EC030
:101690008091E80082FD30C08091E80080FF1DC08D
:1016A0008091F200282F30E008C084918093F100EF
:1016B0003196415050402F5F3F4F4115510519F071
:1016C0002830310590F390E02830310509F491E09D
:1016D0008091E8008E778093E8004115510569F606
:1016E000992359F609C08EB3882361F0853061F0E3
:1016F0008091E80083FD0AC08091E80082FFF3CF6B
:1017000080E0089582E0089583E0089581E00895DF
:10171000EF92FF920F931F93CF93DF939C01009161
:10172000EA021091EB020617170718F4790190E00E
:101730003EC06115710511F08B01F8CF8091E80072
:101740008E778093E80000E010E0F0CF8EB388231E
:1017500009F442C0853009F441C08091E80083FD5E
:101760003FC08091E80082FD31C08091E80080FF99
:101770001EC08091F200C82FD0E00AC0C70168D512
:101780008093F1000894E11CF11C01501040219657
:101790000115110519F0C830D10580F390E02897A4
:1017A00009F491E08091E8008E778093E8000115BC
:1017B000110561F6992351F609C08EB3882361F0B3
:1017C000853061F08091E80083FD0AC08091E800D7
:1017D00082FFF3CF80E005C082E003C083E001C058
:1017E00081E0DF91CF911F910F91FF90EF900895CD
:1017F000BF92CF92DF92EF92FF920F931F93CF93FE
:10180000DF938C01EB016A0158D1B82E8823B9F51A
:1018100021970C0F1D1F2196C114D10439F0F60138
:1018200080819181C81BD90B081B190BEE24FF2462
:1018300024C08091E80085FD16C08091E8008B7778
:101840008093E80064D3C114D10449F0F60180818B
:1018500091818E0D9F1D9183808385E011C02DD1D4
:10186000882359F00DC08091F100F8018083015068
:10187000104021970894E11CF11C2097D1F68B2D84
:10188000DF91CF911F910F91FF90EF90DF90CF905C
:10189000BF900895BF92CF92DF92EF92FF920F9385
:1018A0001F93CF93DF93182F092F7B016A0105D176
:1018B000B82E8823B1F5812F902F9C01E901C11426
:1018C000D10439F0F60180819181E81AF90AC80F34
:1018D000D91F00E010E022C08091E80085FD16C00D
:1018E0008091E8008B778093E80011D3C114D10474
:1018F00049F0F60180819181800F911F918380834F
:1019000085E010C0DAD0882349F00CC08091F10046
:1019100089930894E108F1080F5F1F4FE114F10467
:10192000D9F68B2DDF91CF911F910F91FF90EF9002
:10193000DF90CF90BF900895BF92CF92DF92EF9249
:10194000FF920F931F93CF93DF93182F092F7B01E3
:101950006A01B3D0B82E8823B1F5812F902F9C0156
:10196000E901C114D10439F0F60180819181E81AAE
:10197000F90AC80FD91F00E010E022C08091E800EA
:1019800085FD16C08091E8008E778093E800BFD275
:10199000C114D10449F0F60180819181800F911F1B
:1019A0009183808385E010C088D0882349F00CC0E3
:1019B00089918093F1000894E108F1080F5F1F4FAF
:1019C000E114F104D9F68B2DDF91CF911F910F9186
:1019D000FF90EF90DF90CF90BF9008958F7080932D
:1019E000E9008091EB0081608093EB001092ED00A4
:1019F0006093EC004093ED008091EE00881F8827F3
:101A0000881F08950F931F93CF93DF93062FEC0148
:101A100010E02AC09881992329F16B81E981FA812C
:101A20002C81892F8F70853018F5223010F452E008
:101A300001C056E040E028E030E003C04F5F220FD5
:101A4000331F2E173F07D0F36295660F660F607C39
:101A5000991F9927991F692B4295407F452BBEDF1F
:101A6000882331F01F5F25961017A0F281E001C096
:101A700080E0DF91CF911F910F9108958091E40252
:101A800088238CF403C08EB38823B1F08091E800E2
:101A900082FFF9CF8091E8008B778093E80008956A
:101AA0008EB3882349F08091E80080FFF9CF8091C0
:101AB000E8008E778093E80008954091E40050910B
:101AC000E5002AEF8091EC0080FF23C08091E800C0
:101AD00080FD1DC08EB3882311F482E00895853007
:101AE00011F483E008958091EB0085FF02C081E04E
:101AF00008958091E4009091E5008417950711F313
:101B0000222311F484E008952150AC01DBCF80E062
:101B100008958091E80082FFDDCFF9CF3CD03ED020
:101B20008091D8008F778093D8008091D80080680A
:101B30008093D8008091D8008F7D8093D80084E076
:101B400089BD86E089BD09B400FEFDCF1EBA1092A2
:101B5000E20280E060E042E041DF8091E1008E7FC0
:101B60008093E1008091E20081608093E2008091A7
:101B7000E20088608093E2008091E0008E7F809395
:101B8000E0000895E3E6F0E080818E7F808381E0CD
:101B90008093E302C3CF1092E20008951092E10017
:101BA00008951F920F920FB60F9211242F933F9317
:101BB0004F935F936F937F938F939F93AF93BF9355
:101BC000EF93FF938091E10080FF17C08091E200C6
:101BD00080FF13C08091E2008E7F8093E2008091AD
:101BE000E20080618093E2008091D800806280935F
:101BF000D80019BC1EBA0E94AA018091E10084FF9E
:101C00002FC08091E20084FF2BC084E089BD86E074
:101C100089BD09B400FEFDCF8091D8008F7D8093EF
:101C2000D8008091E1008F7E8093E1008091E200F6
:101C30008F7E8093E2008091E20081608093E200D9
:101C40008091E202882311F084E007C08091E300D4
:101C500087FD02C081E001C083E08EBB0E94A80125
:101C60008091E10083FF21C08091E20083FF1DC0CD
:101C70008091E100877F8093E10082E08EBB10922B
:101C8000E2028091E1008E7F8093E1008091E2008A
:101C90008E7F8093E2008091E20080618093E20079
:101CA00080E060E042E09ADE31D1FF91EF91BF9198
:101CB000AF919F918F917F916F915F914F913F91E4
:101CC0002F910F900FBE0F901F9018951F93DF93C9
:101CD000CF9300D00F92CDB7DEB7E4EEF2E0809163
:101CE000F100819382E0EC3EF807C9F70E943A02C6
:101CF0008091E80083FFF5C08091E4029091E502B5
:101D0000953009F46FC0963040F4913091F19130E4
:101D100070F0933009F0E5C02CC0983009F4B3C0DE
:101D2000993009F4C2C0963009F0DBC07DC080381C
:101D300011F490E014C0823809F0D3C08091E80219
:101D40008F708093E9008091EB0090E025E09695FC
:101D500087952A95E1F7982F91701092E90080916C
:101D6000E800877F8093E8009093F1001092F100E3
:101D700095C0882319F0823009F0B3C08F7182308A
:101D800009F0AFC08091E602882331F52091E80286
:101D90002F7009F4A6C02093E9008091EB0080FF2A
:101DA0001BC0933021F48091EB00806213C08091BE
:101DB000EB0080618093EB0081E090E002C0880F2F
:101DC000991F2A95E2F78093EA001092EA00809129
:101DD000EB0088608093EB001092E9008091E800AE
:101DE000877F5FC0882309F07CC01091E6021F77CF
:101DF0008091E3008078812B8093E3008091E8005C
:101E0000877F8093E8003ADE8091E80080FFFCCF76
:101E10008091E30080688093E300112311F482E055
:101E200001C083E08EBB5DC08058823008F059C08D
:101E30008091E6029091E7026091E802AE014E5F68
:101E40005F4F9E012F5F3F4F0E943102BC01009700
:101E500009F447C08091E800877F8093E8002981DA
:101E6000222321F48A819B81F0DB07C08A819B8138
:101E7000213011F44DDC01C086DB8091E8008B77C6
:101E80008093E8002EC0803861F58091E800877F5C
:101E90008093E8008091E2028093F1008091E80055
:101EA0008E778093E800EADD1CC08823D1F49091FE
:101EB000E6029330B0F48091E800877F8093E800D9
:101EC0009093E202DBDD8091E202882331F480917D
:101ED000E30087FD02C081E001C084E08EBB0E9468
:101EE00043028091E80083FF0AC08091E800877F69
:101EF0008093E8008091EB0080628093EB000F906C
:101F00000F900F90CF91DF911F91089508951F9327
:101F10008EB3882371F01091E9008091EC0010924B
:101F2000E9008091E80083FF01C0D0DE1F701093AC
:101F3000E9001F910895FC018EB3843029F584894E
:101F40009589A689B7890097A105B105E9F0868131
:101F50008F708093E9008091E80082FF15C0809126
:101F6000F200882319F42FEF3FEF04C08091F100B5
:101F7000282F30E08091F200882341F48091E8001E
:101F80008B778093E80002C02FEF3FEFC9010895DF
:101F90000895FC018EB3843019F584899589A6894A
:101FA000B7890097A105B105D9F081818F70809321
:101FB000E9008091F2008823A9F09091E8008091D7
:101FC000E8008E778093E80095FD0CC076DD982FB1
:101FD000882349F48091E8008E778093E80003C05D
:101FE00092E001C090E0892F0895FC018EB3843007
:101FF00091F484899589A689B7890097A105B105CF
:1020000051F081818F708093E9008091E80080FF1A
:1020100002C0CF01BECF08951F93FC01162F8EB3CF
:102020008430E1F484899589A689B7890097A10550
:10203000B105A1F081818F708093E9008091E80063
:1020400085FD08C08091E8008E778093E80035DD3B
:10205000882329F41093F10080E001C082E01F91F1
:102060000895CF93DF93EC014096FC018BE0DF01F4
:102070001D928A95E9F782E08C83898783E08E87B9
:10208000CE01019661E0BEDC882371F0CE01069698
:1020900061E0B8DC882341F0CE010B9661E0B2DC50
:1020A000882319F081E001C080E0DF91CF9108958D
:1020B000CF93DF93EC018091E80083FFA4C0888177
:1020C00090E02091E8023091E9022817390709F0E1
:1020D0009AC08091E502813269F0823220F4803228
:1020E00009F091C03CC0823209F46BC0833209F020
:1020F0008AC07BC08091E402813A09F084C080915B
:10210000E800877F8093E8008091E80080FFFCCFA3
:102110008C899D89AE89BF898093F100292F3A2F40
:102120004B2F55272093F1009D01442755272093DD
:10213000F1008B2F9927AA27BB278093F100888D68
:102140008093F100898D8093F1008A8D8093F10056
:102150008091E8008E778093E80090DC54C08091F5
:10216000E402813209F04FC08091E800877F8093BC
:10217000E80004C08EB3882309F445C08091E800CC
:1021800082FFF8CF8091F1009091F1002091F10051
:102190003091F1008C8B9D8B2E8B3F8B8091F100C9
:1021A000888F8091F100898F8091F1008A8F8091D2
:1021B000E8008B778093E80061DCCE010E94EC019F
:1021C00022C08091E4028132F1F48091E800877F9F
:1021D0008093E80053DC8091E6029091E702998BAE
:1021E000888BCE010E94AC010EC08091E402813246
:1021F00051F48091E800877F8093E8003FDCCE01B6
:102200006091E602C5DEDF91CF910895A1E21A2E1A
:10221000AA1BBB1BFD010DC0AA1FBB1FEE1FFF1F8A
:10222000A217B307E407F50720F0A21BB30BE40BDA
:10223000F50B661F771F881F991F1A9469F7609521
:102240007095809590959B01AC01BD01CF010895DB
:10225000F999FECF92BD81BDF89A992780B508956E
:10226000262FF999FECF92BD81BDF89A019700B44F
:10227000021639F01FBA20BD0FB6F894FA9AF99AEF
:082280000FBE0895F894FFCF92
:102288000083100000010410000001820800000112
:10229800000000000000000000000009023E0002EB
:1022A8000100C032090400000102020100052400F7
:1022B800100104240206052406000107058203080C
:1022C80000FF09040100020A0000000705040210CB
:1022D800000507058302100005090220000101001E
:1022E800C0320904000002FF000000070582024016
:1022F800000A0705020240000A1C033000300030C3
:102308000032003000300030003100320033003439
:10231800003500000000004156524953505F4D4BB4
:1023280032008001008101009001009101019201B9
:10233800189401219803069E0301A10100A403003B
:02234800010092
:00000001FF
